:020000009E2F31
:10000600031C0B288312031305148514851010286E
:0C001600831203130510851485100800E8
:1000220083120313051586156400E6016608073C72
:10003200031C2028E50CE5130320E60A1728051106
:10004200E60166080F3C031C312808306602031CD7
:100052002B280515E90CE80CE9130320E60A2228EF
:10006200E6016608073C031C3B28E70CE713032064
:10007200E60A3228E6016608073C031C4528EA0D19
:100082006A100320E60A3C2805110330FC00973071
:10009200FD00FD0B4A28FC0B4A2800000000051554
:0400A20086150800B7
:1000A6008316031398185928000053284108831211
:0400B60099000800A5
:1000BA0083120313FB01FA01F9018030F800F10CF5
:1000CA00F00C031C71287408F90775080318750FDA
:1000DA00FA070318FB0A0310F01F79287408FA07B5
:1000EA0075080318750FFB07FB0CFA0CF90CF80CD2
:1000FA00031C64287B08F3007A08F2007908F100EF
:06010A007808F000080077
:10011000831203137008F100F0010830FC0071082D
:10012000F40C03189728FC0B9028F10100340310FD
:100130009C28F40C0318F107F10CF00CFC0B992827
:020140000800B5
:100142008316031398169030831298008316861430
:10015200061183128C1EB0281A08F000AA28080083
:0E016200831203136D088A006C0882000800E7
:1001700083120313FB01FA01F901F801A001730DC9
:10018000F80D7408F8027508031C750FF90276085B
:10019000031C760FFA027708031C770FFB0200019D
:1001A000031C0130A002F30D0730FC00730DF80DA5
:1001B000F90DFA0DFB0DA00D7408731CF128F8025F
:1001C0007508031C750FF9027608031C760FFA02F6
:1001D0007708031C770FFB020001031C0130A0020B
:1001E0000229F80775080318750FF9077608031830
:1001F000760FFA0777080318770FFB07000103183B
:100200000130A007F30DFC0BD628720DF80DF90D87
:10021000FA0DFB0DA00D7408731C2029F802750857
:10022000031C750FF9027608031C760FFA02770893
:10023000031C770FFB020001031C0130A0023129CF
:10024000F80775080318750FF90776080318760F75
:10025000FA0777080318770FFB070001031801302E
:10026000A007F20D0730FC00720DF80DF90DFA0D24
:10027000FB0DA00D7408721C4F29F8027508031CB1
:10028000750FF9027608031C760FFA027708031C33
:10029000770FFB020001031C0130A0026029F80760
:1002A00075080318750FF90776080318760FFA0713
:1002B00077080318770FFB07000103180130A00728
:1002C000F20DFC0B3429710DF80DF90DFA0DFB0D33
:1002D000A00D7408721C7E29F8027508031C750FA6
:1002E000F9027608031C760FFA027708031C770FD1
:1002F000FB020001031C0130A0028F29F8077508DA
:100300000318750FF90776080318760FFA077708B0
:100310000318770FFB07000103180130A007F10D48
:100320000730FC00710DF80DF90DFA0DFB0DA00D55
:100330007408711CAD29F8027508031C750FF902C9
:100340007608031C760FFA027708031C770FFB026E
:100350000001031C0130A002BE29F807750803182C
:10036000750FF90776080318760FFA077708031850
:10037000770FFB07000103180130A007F10DFC0BFC
:100380009229700DF80DF90DFA0DFB0DA00D7408F2
:10039000711CDC29F8027508031C750FF902760838
:1003A000031C760FFA027708031C770FFB0200018B
:1003B000031C0130A002ED29F80775080318750F1A
:1003C000F90776080318760FFA0777080318770FEE
:1003D000FB07000103180130A007F00D0730FC00F7
:1003E000700DF80DF90DFA0DFB0DA00D7408701CC1
:1003F0000B2AF8027508031C750FF9027608031C16
:10040000760FFA027708031C770FFB020001031C2A
:100410000130A0021C2AF80775080318750FF907A8
:1004200076080318760FFA0777080318770FFB078B
:10043000000103180130A007F00DFC0BF029701823
:100440002F2A7408F80775080318750FF90776083E
:100450000318760FFA0777080318770FFB070800D1
:100460009A01981718168C1E332A1A08EB00981C4C
:08047000080018120800080042
:1004780083160313C00183126E0884000008EF007E
:100488006F08003A0319552A6F088316C1005320D4
:100498008316C00A400883126E0784000008EF0024
:0404A800442A0800DA
:1004AC00831203132230FC00F801F901FA01FB015D
:1004BC00FC0303198C2A0310FB0CFA0CF90CF80C36
:1004CC00F30CF20CF10CF00C031C5E2AFC03031968
:1004DC007E2A7408F80775080318750FF907760853
:1004EC000318760FFA0777080318770FFB07622AB1
:1004FC007408F80775080318750FF90776080318C0
:0E050C00760FFA0777080318770FFB07080031
:10051A00293083120313E5009B30E800B230E9006A
:10052A001030E700EA0111202830E500B030E80079
:10053A001630E9002D08E700EA0111200616861296
:06054A00061386130800F1
:10055000831203130618B02A2130EE003C22B32A7E
:080560002530EE003C220800EA
:100568000030831203136402031DC42A153063028A
:10057800031DC42A35306202031DC42AAF3061024C
:100588000318D72A6408013C031DD42A6308D93C00
:10059800031DD42A6208053C031DD42A6108C03C07
:1005A8000318D72AB42A00306402031DE52A15303F
:1005B8006302031DE52A5C306202031DE52AC03090
:1005C8006102031C002B6408003C031DF52A630824
:1005D800213C031DF52A6208913C031DF52A610898
:1005E800BF3C031C002B3508B00006128612061308
:1005F80086132030B3009A2C00306402031D0E2BA2
:1006080021306302031D0E2B91306202031D0E2B55
:10061800C0306102031C292B6408003C031D1E2BFB
:1006280063082D3C031D1E2B62089F3C031D1E2BD7
:100638006108AF3C031C292B3408B000061686124B
:10064800061386131030B3009A2C00306402031D81
:10065800372B2D306302031D372BC6306202031D72
:10066800372BC0306102031C522B6408003C031D69
:10067800472B6308443C031D472B6208833C031D3A
:10068800472B61080F3C031C522B5B08B000061671
:100698008612061386131030B3009A2C00306402B9
:1006A800031D602B44306302031D602BAA306202D5
:1006B800031D602B20306102031C7B2B6408003C67
:1006C800031D702B63085B3C031D702B6208663C9E
:1006D800031D702B61086F3C031C7B2B5C08B0006A
:1006E80006128616061386130830B3009A2C0030BB
:1006F8006402031D892B5B306302031D892B66305E
:100708006202031D892B70306102031CA42B64084C
:10071800003C031D992B6308893C031D992B620833
:100728002D3C031D992B61082F3C031CA42B590851
:10073800B00006128616061386130830B3009A2CEA
:1007480000306402031DB22B89306302031DB22BF3
:100758002D306202031DB22B30306102031CCD2BF9
:100768006408003C031DC22B6308B63C031DC22B62
:100778006208F33C031DC22B6108EF3C031CCD2B20
:100788005A08B00006168616061386130430B300FE
:100798009A2C00306402031DDB2BB6306302031D64
:1007A800DB2BF3306202031DDB2BF0306102031CEC
:1007B800F62B6408013C031DEB2B63080A3C031D60
:1007C800EB2B6208E03C031DEB2B61084F3C031C3C
:1007D800F62B5F08B000061286120617861304303F
:1007E800B3009A2C01306402031D042C0A30630202
:1007F800031D042CE0306202031D042C50306102FA
:10080800031C1F2C6408013C031D142C6308313C95
:10081800031D142C6208053C031D142C6108EF3CD1
:10082800031C1F2C6008B0000616861206178613D4
:100838000430B3009A2C01306402031D2D2C313092
:100848006302031D2D2C05306202031D2D2CF03090
:100858006102031C482C6408013C031D3D2C6308FD
:100868005E3C031D3D2C6208CC3C031D3D2C6108F9
:10087800AF3C031C482C5D08B0000612861606170C
:1008880086130430B3009A2C01306402031D562CE1
:100898005E306302031D562CCC306202031D562CB9
:1008A800B0306102031C712C6408013C031D662CE6
:1008B80063088C3C031D662C6208933C031D662C60
:1008C80061086F3C031C712C5E08B0000616861682
:1008D800061786130430B3009A2C01306402031DF6
:1008E8007F2C8C306302031D7F2C93306202031D22
:1008F8007F2C70306102031C9A2C6408013C031D94
:100908008F2C6308D83C031D8F2C6208DE3C031D26
:100918008F2C6108B03C031C9A2C5108B0000612B9
:100928008612061386170430B3009A2C051EC72CAE
:100938001030F4002730F500F601F7016108F000E7
:100948006208F1006308F2006408F3007408F0021A
:100958007508031C750FF1027608031C760FF20266
:100968007708031C770FF3023308F400F501F6014A
:10097800F70156227008E1007108E2007208E300EE
:100988007308E400112D5208013A0319D02C4C08C1
:10099800013A0319D02CFB2C8C30F4002330F500DD
:1009A800F601F7016108F0006208F1006308F2003F
:1009B8006408F3007408F0027508031C750FF1024F
:1009C8007608031C760FF2027708031C770FF302F0
:1009D8003308F400F501F601F70156227008E1002A
:1009E8007108E2007208E3007308E400112D610841
:1009F800F0006208F1006308F2006408F3003308AD
:100A0800F400F501F601F70156227008E1007108BB
:100A1800E2007208E3007308E4001030F4002730A5
:100A2800F500F601F7016108F0006208F1006308BB
:100A3800F2006408F300B8207008AE007108AF0037
:100A48000030F200F300A030F4008630F5000130E9
:100A5800F6000030F70056227008CD007108CE006D
:100A68007208CF007308D0000A30F400F501F601CF
:100A7800F701B8207008CD007108CE007208CF00C9
:100A88007308D0006108F4006208F5006308F600F6
:100A98006408F7007008F4027108031C710FF5026E
:100AA8007208031C720FF6027308031C730FF70217
:100AB8007408D5007508D6007608D7007708D800DE
:100AC8000A30F000F101F201F30156228830F400F7
:100AD8000130F500F601F701B8207008B10071087F
:100AE800B2002E08E8002F08E9007008EA000800A4
:100AF8006400293083120313EE003C2230226B0875
:100B0800493A031D892D30228A2D7C2D6B08463ADF
:100B1800031D922D302230223022932D7C2DE601A8
:100B28006608203C031CA02D30226608A03E8400E5
:100B38006B088000E60A942D83163708313A031DA6
:100B4800A82D83120512AA2D8312051683163808BC
:100B5800353A031DB32D01308312D200B52D83120F
:100B6800D20183163808343A031DBE2D0130831292
:100B7800CC00C02D8312CC01831640083B3A031DDC
:100B8800C82D83128515CB2D831285118D22303007
:100B9800831620028312BE00BF01031CBF0300306E
:100BA800BF1BFF30C000C1003E08F0003F08F10045
:100BB8004008F2004108F3008030F4009630F50058
:100BC8009830F6000030F70056227008BE00710811
:100BD800BF007208C0007308C100303083162102BC
:100BE8008312C200C301031CC3030030C31BFF30C0
:100BF800C400C5004208F0004308F1004408F200B0
:100C08004508F3004030F4004230F5000F30F6009C
:100C18000030F70056227008C2007108C30072083D
:100C2800C4007308C5003030831622028312B60050
:100C3800B701031CB7030030B71BFF30B800B90079
:100C48003608F0003708F1003808F2003908F300D8
:100C5800A030F4008630F5000130F6000030F700CF
:100C680056227008B6007108B7007208B8007308F9
:100C7800B9003030831623028312BA00BB01031C6B
:100C8800BB030030BB1BFF30BC00BD003A08F000BE
:100C98003B08F1003C08F2003D08F3001030F40076
:100CA8002730F500F601F70156227008BA007108DE
:100CB800BB007208BC007308BD00303083162402E4
:100CC800F000F101031CF10370088312C8007108D9
:100CD800C900E830F4000330F5005D207008C80052
:100CE8007108C900303083162502F000F101031C99
:100CF800F10370088312CA007108CB006430F40055
:100D08000030F5005D207008CA007108CB00303053
:100D180083162602F00070088312C6000A30F40019
:100D280088207008C6003030831627028312C70057
:020D38000800B1
:100D3A00831203133E08F0003F08F1004008F20056
:100D4A004108F3004208F00743080318430FF1076C
:100D5A0044080318440FF20745080318450FF30720
:100D6A003608F00737080318370FF1073808031851
:100D7A00380FF20739080318390FF3077008F4001F
:100D8A007108F5007208F6007308F7003A08F407CC
:100D9A003B0803183B0FF5073C0803183C0FF607FE
:100DAA003D0803183D0FF7074808F0004908F1000D
:100DBA00F201F3017408F00775080318750FF107BB
:100DCA0076080318760FF20777080318770FF307E8
:100DDA004A08F4004B08F500F601F7017008F40719
:100DEA0071080318710FF50772080318720FF607D6
:100DFA0073080318730FF7074608F000F101F201B0
:100E0A00F3017408F00775080318750FF1077608DF
:100E1A000318760FF20777080318770FF3074708C6
:100E2A00E100E201E301E4017008E1077108031837
:100E3A00710FE20772080318720FE30773080318A9
:060E4A00730FE40708002D
:100E50000730831203139F00831685010330860039
:100E6000831205118510051086110516851582302F
:100E7000FC00DD30FD00FD0B3B2FFC0B3B2F000089
:100E800000008511D201CC01D301D4018B30B50013
:100E90009330B4009B30DB00D330DC00DB30D90072
:100EA000F330DA00FB30DF00F730E000F730DD0030
:100EB000FF30DE00FF30D1000C308316990018158A
:100EC000A1208230FC00DD30FD00FD0B652FFC0B06
:080ED000652F0000000008007E
:100ED800B1208A110A128000840AEC0A0319ED0A6B
:080EE800F003031D6C2F08004C
:100EF000293083120313E5003008003EE800B230C9
:100F00000318013EE9001030E7003108EA00112023
:100F1000640005118514051086112830E5002E089F
:100F2000E8002F08E9002D08E7003108EA00112049
:0C0F3000640005118514051086110800EE
:100F3C00543083120313A1005830A2003B30A3009D
:100F4C00A4015230A5005830A6003B30A700A801E0
:100F5C004930A9004630AA003B30AB00AC01AA30A6
:100F6C00AD00282764008D227C25A822B4229D2662
:060F7C007827BA2FC02FF8
:02400E0025216A
:00000001FF
